S31508001800C0090020D9180008E7180008E9180008D8
S3150800181000000000000000000000000000000000BA
S315080018200000000000000000000000000119000888
S3150800183000000000000000000319000845360008F3
S315080018405D4300080719000807190008071900086A
S31508001850071900080719000807190008FD260008D7
S31508001860071900089924000807190008071900082D
S31508001870071900080719000807190008B1380008F1
S3150800188005390008000000000000000007190008DC
S3150800189000000000071900080719000807190008C2
S315080018A0000000000719000807190008853C000811
S315080018B007190008071900080719000800000000A2
S315080018C0EE11AA550348854600F0ECFA0048004791
S315080018D0B5550008C00900200B4880F308880B4856
S315080018E080470B480047FEE704207146084202D0AD
S315080018F0EFF3098001E0EFF30880714603F02AFD53
S31508001900FEE7FEE7FEE7FEE7C009002045380008C7
S31508001910C518000830B50B460146002020220124D0
S3150800192009E00D46D5409D4205D31D469540491B05
S315080019302546954040191546521E002DF1DC30BD4E
S3150800194070B500242546002801DA01244042002902
S3150800195001DA01254942FFF7DDFFAC4200D04042DB
S31508001960002C00D0494270BD03460B439B0703D0A9
S3150800197009E008C9121F08C0042AFAD203E00B7846
S31508001980491C0370401C521EF9D27047D2B201E0BE
S315080019900270401C491EFBD270470022F6E710B5BC
S315080019A013460A4604461946FFF7F0FF204610BDBF
S315080019B0F8B502464A40D40F42004B0052085B086D
S315080019C09A4202D20246084611464A0023D0C30D5F
S315080019D04A00DDB2120EAD1A202D35DA490201266B
S315080019E0490AF6058A19002C00D0524220214F1BBD
S315080019F01146B9402A411018C20D9A4221D0002C2E
S31508001A0017D0012D08DCDA05801AD20F8019D20703
S31508001A10DBB200F0ACF9F8BDDA05801A0123400004
S31508001A201B06C01880185A428018CA0F104349006E
S31508001A3007E04908C2071143DA05801A80194008E9
S31508001A40801800F08CF9F8BD61000122511A001BBC
S31508001A50F7E70122D2075140AAE70122D2075040F0
S31508001A60A6E7024670B54A40D30FDB0740002DD0E3
S31508001A704A002AD0010E140E091900021202400A61
S31508001A80520A8418E50104465443000A120A2E0431
S31508001A905043A4194219200CC543AA18120C012553
S31508001AA07F39521CAD0352191204240400D0521C6B
S31508001AB0104301D44000491EC2B20C06C0092018C2
S31508001AC0401C4008802A02D003E0002070BD400870
S31508001AD04000002900DA0020184370BD70B50246A0
S31508001AE04A40D50F40004A00ED0740085208002832
S31508001AF014D0002A12D0C40DD30D41020120C0050E
S31508001B005202490A520AE41A091812187D349142F7
S31508001B1001D3641C00E04900002C01DA002070BDE6
S31508001B200023914201D3891A03434008490000283B
S31508001B30F7D100290AD0914202D10121C90705E04F
S31508001B40914201D2012101E00121C943E005C018F3
S31508001B50401900F004F970BDF0B51FB488B00B99B0
S31508001B600998002448400999C00F49004908099175
S31508001B70C0070B990090490049080B9109990898E4
S31508001B80A646084303D00B990A98084303D10020B8
S31508001B9001460DB0F0BD099801244000420D4800E9
S31508001BA0410D099824050003000B204309900B9862
S31508001BB00003000B20430B9050181A4940180022C6
S31508001BC001901446104601E0032801DA034600E0B6
S31508001BD003239C46C11A0AAE0AE05F0008ADED5B16
S31508001BE04F00F75B7D430027AA187C415B1E491C02
S31508001BF06145F2DD410004AB5A522104120C0A4336
S31508001C00240C401C0828DFDB0198029000997046D6
S31508001C1001910090059B049A0799069800F0EEF842
S31508001C20B7E700000DFCFFFF10B50022962311460A
S31508001C3000F09DF810BD410040020122400AD2057D
S31508001C40090E80187F2901DA00207047962903DCDF
S31508001C509622511AC8407047963988407047000046
S31508001C604A0009030123090B1B051943094B10B543
S31508001C70520D9A4201DA002010BD064B34339A42BF
S31508001C8003DC9A1A00F05AF810BD03495118884027
S31508001C9010BD0000FF030000CDFBFFFFC20FD207F7
S31508001CA0400040080BD0C10D0723DB01C9184002CC
S31508001CB00905400A1143C20840071143704700202E
S31508001CC00146704710B5002904DB0124E4074042A9
S31508001CD08C412146002B04DB1C460123DB075242BC
S31508001CE0A3418B4200D1824210BD000010B50029E5
S31508001CF004DB0124E40740428C412146002B04DB27
S31508001D001C460123DB075242A341994200D1904267
S31508001D1010BD00000122D207002800DB101A002996
S31508001D2000DB511A814270470122D207002800DBE6
S31508001D30101A002900DB511A8842704710B5202A6C
S31508001D4004DB0846203AD040002110BD0B46D3409C
S31508001D50D0402024A21A91400843194610BD0029F4
S31508001D6004DA401C490001D140084000704770B4AD
S31508001D700024050C05D11024000402D1002922D024
S31508001D801124050E01D108340002050F01D1241DC6
S31508001D900001850F01D1A41C8000002801DB641C0A
S31508001DA04000002908D020252E1B0D46F540A140ED
S31508001DB000D00121294308431B1B0106DB1D000A2D
S31508001DC0002B02DA002070BC7047DB051818801853
S31508001DD00029F8DA401C4900F5D170BC40084000DB
S31508001DE0704710B5002B08DA0024401C6141921890
S31508001DF05B411A4301D14008400010BDF0B51FB43D
S31508001E0082B005460C0003D0084602F0E3FA02E069
S31508001E1002F0E0FA2030024600902146284600F0FB
S31508001E2053F8049B059A04460F4618431143084382
S31508001E3003D12046394607B0F0BD1846104317D0DF
S31508001E40009840210A1A18460599FFF777FF0546B4
S31508001E500E46009A0599049800F036F8084301D012
S31508001E60012000E00020C11705430E432C433743E9
S31508001E7000990E986305401A7905E40A0A3000228B
S31508001E800C43FD0A002802DA00200146D3E70105C3
S31508001E90101969410C9C0D9D00196941FFF7A1FFB6
S31508001EA0C9E70000064C0125064E05E02046E36812
S31508001EB007C82B4398471034B442F7D3FFF706FDFB
S31508001EC0586300087863000810B5202A04DB014629
S31508001ED0203A9140002010BD914020239C1A0346C9
S31508001EE0E3401943904010BD10B50446002C08D1B4
S31508001EF001210920C00600F05FFE002000F0AAF8C4
S31508001F0052E0012C05D102210920C00600F054FE3A
S31508001F104AE0022C05D104210920C00600F04CFE37
S31508001F2042E0032C05D108210920C00600F044FE32
S31508001F303AE0042C05D110210920C00600F03CFE29
S31508001F4032E0052C05D120210920C00600F034FE18
S31508001F502AE0062C05D140210920C00600F02CFEF7
S31508001F6022E0072C05D180210920C00600F024FEB6
S31508001F701AE0082C04D101210D4800F01DFE13E0DB
S31508001F80092C04D102210A4800F016FE0CE00B2C9D
S31508001F9004D11021064800F00FFE05E00C2C03D1F1
S31508001FA08021034800F008FE204600F053F810BDD3
S31508001FB0000400487FB5002000900190029003902D
S31508001FC000241BE000250CE0E8000E4940186100DB
S31508001FD0405AA1006A4651584018A1005050681C42
S31508001FE085B2142DF0DBA1006A4650581421FFF77C
S31508001FF091FC6100044A5052601C84B2042CE1DB57
S315080020007FBD0000180400207001002000B587B0CD
S3150800201001A800F0ADF80121480201F089F9002075
S315080020200190302002900120400203900020069083
S31508002030059001A9064800F031F80121044800F08E
S3150800204021F80121024800F011F807B000BD000090
S315080020500024014010B50446072300222146024801
S3150800206000F038F810BD000000240140002904D013
S31508002070426801231A43426003E04268520852004C
S3150800208042607047002904D0826808231A43826098
S3150800209003E0826808239A438260704742680B4BC4
S315080020A01A4042600B684A681A4343681A434260FA
S315080020B08268074B1A4082600B694A691A438B6823
S315080020C01A4383681A438260704700000FBCFFFFFB
S315080020D08FF1F9FFF0B504460D4616461F463F0731
S315080020E03F0F2B46082B0FD91B071B0F083B606FAA
S315080020F09A000F21914088436067606F99003A46BD
S315080021008A40104360670BE0206F9A000F219140C8
S3150800211088432067206F99003A468A401043206713
S31508002120E0680121A9408843E060E0680121A940F0
S315080021300843E06001208003054203D0012000F037
S315080021401FF806E00120C003054202D0012000F076
S3150800215017F8F0BD002905D08268FF2301331A431A
S31508002160826004E08268FF2301339A4382607047E5
S31508002170002101604160816001730161416170471E
S31508002180002806D0064949680C221143044A5160C2
S3150800219005E0034949680C229143014A516070479A
S315080021A00024014010B507480078002806D0FFF73C
S315080021B001FF00200349087000F046FD7E2002F06A
S315080021C0D9F810BD78010020FFB583B00C460294FB
S315080021D000200190002726E000261CE0721C0399C7
S315080021E051430846791CFFF795FB0546A54201D9D8
S315080021F0281B00E0601B05460298A84204D90295F0
S3150800220005980670069807700298002802D10120E2
S31508002210019002E0761C402EE0D300BF019800280A
S3150800222000D002E07F1C042FD6D300BF029807B067
S31508002230F0BD000000BF00BF00BF00BF00BFBFF376
S315080022404F8F00BF00BF00BF06480749C86000BFE0
S3150800225000BF00BFBFF34F8F00BF00BF00BF00BF66
S3150800226000BFFDE70400FA0500ED00E010B500F038
S3150800227001F810BD10B523480078002817D1224868
S3150800228001F0DCF801283CD11F480078002838DD29
S315080022901D480078402834DC01F0C7FC1B4908605B
S315080022A001201849087000201949087029E0164AC3
S315080022B017490978491C501801F0C0F8012816D1A9
S315080022C013480078401C124908700F4800780978AE
S315080022D0884216D100200B4908700B484078FF2821
S315080022E00FD10B48007802280BD1FFF7A3FF01F0A6
S315080022F09CFC064909686431884202D900200149D4
S31508002300087010BD290100209C0300202C01002024
S315080023102801002078B50246002327E0002020E0A7
S315080023208400155B441CA400145BA54218DD8400D8
S31508002330A5182E886C4626806D8865808400A518A9
S31508002340441CA400A41826882E8064886C80441C2B
S31508002350A400A5186C4624882C806C4664886C807A
S31508002360401C4C1EE41A8442DADC5B1C4C1E9C4260
S31508002370D4DC78BD10B586B004460121880300F088
S31508002380D7FF0121880400F0B3FF03221146224833
S3150800239000F0FEFB032204211F4800F0F9FB01A808
S315080023A001F013FD01943021684601810021418125
S315080023B0818101821821C18101A9184801F0C2FC56
S315080023C00121164801F09DFC05A800F035FC0821FE
S315080023D068468182012181751821C17505A90E48B3
S315080023E000F08CFB1021684681824821C17505A939
S315080023F0094800F083FB1B216846017003214170E0
S315080024000121817000F022FF01220221034801F018
S315080024108EFC06B010BD00000004004800380140DC
S3150800242070B502460B46FF25FF2408E01178521CBA
S3150800243069400748405C604005460648445C1846C3
S315080024405E1EB3B20028F1D12802204370BD0000F9
S315080024505861000858620008014600220D4B1A61AF
S31508002460CA005A6100229A6105221A6100BF094A08
S315080024701069C207D20F03D0012212041042F6D007
S31508002480044A126952085200024B1A6100229A61E4
S315080024907047000000E000E010B500210848FFF78B
S315080024A059FE022000F052F8012006490870010280
S315080024B00920C00600F0BCFB02F00CF810BD0000B5
S315080024C0002401404401002000B589B001210846D6
S315080024D000F00EFF1A4800F045F801A800F08EF843
S315080024E01848019018480290002168460173042094
S315080024F0049068460175802141754900C1828900AA
S31508002500018320218176090281830021C183018408
S3150800251001A90B4800F04CF80121094800F01CF805
S3150800252001220221064800F039F80921684601709F
S31508002530022141700121817000F088FE09B000BDBA
S315080025400800024000240140E003002001494860D9
S3150800255070470000000002400268520852000A4311
S315080025600260704710B504462068400840002060A5
S31508002570002020606060A060E060E1B2084608388C
S315080025800521FFF7C7F901460F2088400249496827
S3150800259008430149486010BD00000240002A03D0E4
S315080025A003680B43036002E003688B4303607047CC
S315080025B010B50A7A8B7D1A430B7C1A434B7C1A4357
S315080025C04B8A1A438B8A1A430B8B1A434B8B1A4333
S315080025D00368094C23401A43026002680123DB039F
S315080025E09A438B8B1A430260CA6842600A68826003
S315080025F04A68C26010BD00000F80FFFF002101601D
S3150800260041600172C16001744174418281828175A1
S31508002610018341838183704770B506460C4621467F
S315080026200A4800F00DFA0546002D01D1401E70BD7E
S315080026300648854202D10648051B00E02D1B2246A6
S3150800264029463046FFF790F92046F0E700F40008DF
S3150800265000FC000870B506460C4621460A4800F0FC
S31508002660EFF90546002D01D1401E70BD064885428A
S3150800267002D10648051B00E02D1B22462946304696
S31508002680FFF772F92046F0E700F0000800F80008A6
S3150800269070B506460C4621460A4800F0D1F90546AB
S315080026A0002D01D1401E70BD0648854202D106485C
S315080026B0051B00E02D1B224629463046FFF754F934
S315080026C02046F0E700F800080000010870B5054646
S315080026D00C4622460249284600F073F9204670BD8A
S315080026E000F4000870B505460C46224602492846FD
S315080026F000F067F9204670BD00F0000810B50248E2
S3150800270000F004F810BD000020800000014948616F
S3150800271070470000000401401CB5684600F0A9F89F
S315080027200F21002000F07CF80120C0030090002152
S3150800273068460171102141710121817100F010F87C
S315080027400521002000F06CF8202000900021684642
S315080027500171102141710121817100F001F81CBD40
S315080027608179002948D02D490968026891432B4A86
S3150800277011601146496802689143284A51600179F7
S31508002780002906D11146096802681143234A1160D7
S3150800279005E02249496802681143204A51601F49E9
S315080027A08968026891431D4A91601146C9680268A2
S315080027B091431A4AD160417910290CD1114689688A
S315080027C002681143154A91601146C96802681143A7
S315080027D0124AD16020E04179082906D10F49896853
S315080027E0026811430D4A916016E00C49C9680268EF
S315080027F011430A4AD1600FE00179002906D1074939
S31508002800096802689143054A116005E00349496869
S3150800281002689143014A5160704700000004014074
S3150800282010B50D4A8B109B00D3588A07140F0F2238
S31508002830A2409343084A8C10A40013518B109B00A6
S31508002840D2588B071C0F0346A3401A43024B8C1021
S31508002850A4001A5110BD00000800014008B5072160
S3150800286068460170022141700121817000F0EEFC7A
S3150800287008BD0021016001710C214171002181719F
S315080028807047000010B5044608480069022108434D
S31508002890064908610846446100694021084303491E
S315080028A00861034800F00AF910BD00000020024044
S315080028B0FF0F00000B48C068C007C00F01D00120F9
S315080028C070470848C0680421084201D00220F7E78B
S315080028D00448C0681021084201D00320F0E704200C
S315080028E0EEE7000000200240034800698021084303
S315080028F001490861704700000020024030B50446CF
S315080029000D460548006901210843034908612580E9
S315080029100F2000F0D3F830BD0020024010B57E200D
S3150800292001F028FD064800F00FF87E2001F022FD90
S31508002930044800F009F87E2001F01CFD10BD0000D7
S3150800294000F4000800F0000810B5044600F0AAF8E4
S315080029502046FFF797FFFFF7C7FF10BD70B5034680
S315080029600125002208E050001C5A0748844201D07D
S31508002970002506E0501C82B2CE0F761876109642D5
S31508002980F1DC00BF284670BDFFFF0000F8B505461C
S315080029900E46144600F086F87E2001F0EBFC002770
S315080029A007E029883046FFF7A9FFB61CAD1C781C3E
S315080029B087B2E10F09194910B942F2DCFFF794FF13
S315080029C0F8BDF8B507460C4615462946204600F0D8
S315080029D037F80646002E0DD12046FFF7B5FF012031
S315080029E080022018FFF7B0FF2A4621463846FFF72F
S315080029F0CDFF24E0012080022018401BB0420AD1F6
S31508002A00012080022018FFF79FFF2A4631463846E4
S31508002A10FFF7BCFF13E00120C0022018401BB0429C
S31508002A2008D12046FFF790FF2A4631463846FFF779
S31508002A30ADFF04E02A4631463846FFF7A7FFF8BD42
S31508002A40F8B505460E462F46E807C00F01D000BF69
S31508002A50FEE731460120C002FEF772FF002901D0C9
S31508002A6000BFFEE700240BE02046704347193146B5
S31508002A703846FFF773FF012800D108E0601C84B2CE
S31508002A8031460120C002FEF75BFFA042ECDC00BF26
S31508002A9031460120C002FEF753FFA04200D10027AD
S31508002AA03846F8BD024803494860034848607047FD
S31508002AB02301674500200240AB89EFCD10B50246D9
S31508002AC000BFFFF7F7FE0346521EFF2400E0641E10
S31508002AD0002CFCD1012B01D1002AF2D1064800694D
S31508002AE077218843044908613420C860002A01D147
S31508002AF0052010BD1846FCE700200240F8B502463E
S31508002B00CD782F073F0FCD781026354201D08D7826
S31508002B102F431446002010E085062B0E0D8801264B
S31508002B208640354207D025680F269E40B5433E4667
S31508002B309E4035432560451CE8B20828ECDB141D89
S31508002B400D882D120095002010E085062B0E012514
S31508002B508540009E354207D025680F269E40B5431E
S31508002B603E469E4035432560451CE8B20828ECDB06
S31508002B70CD78282D04D155690E883543556106E070
S31508002B80CD78482D03D115690E8835431561F8BDF2
S31508002B9070B54D07EB0E082902DA0546203501E027
S31508002BA0054624352C460F269E402568B54316460D
S31508002BB09E403543256070BD38B504460D4609204C
S31508002BC0C006844203D10121480400F091FB114854
S31508002BD0844203D10121000200F08AFB0E48844298
S31508002BE003D10121000200F083FB0C48844203D183
S31508002BF00121080500F07CFB684600F01DF86846D0
S31508002C000580012181700021C17069462046FFF7C1
S31508002C1075FF38BD0004004800080048000C00484D
S31508002C2002469068084201D0012070470020FCE760
S31508002C3041617047016170470021C9430180022143
S31508002C4081700421C1707047F0B587B000200690E6
S31508002C500590049003907E2001F08CFB002611E07D
S31508002C607100BB4A505AFEF7DFFF0546B949FEF721
S31508002C7035FF0446B849FEF7F4FEB100B74A50508E
S31508002C80701C86B2042EEBDBB44A51689068FEF7D6
S31508002C90E0FE0446B249FEF721FF0690AF494868B0
S31508002CA00699FEF71BFFAF490860AF48807B0028EE
S31508002CB03FD1AD4910318889FEF7B6FFAA491031D0
S31508002CC00190C888FEF7B0FFA8490090FEF706FFF6
S31508002CD007460199FEF7C5FE0546A549FEF7FEFE1D
S31508002CE00446A14910318889FEF79EFF0746A04988
S31508002CF0FEF7F4FE05469B4801682846FEF7ADFE3A
S31508002D0021460290FEF7EAFE049097491031488959
S31508002D10FEF78AFF05460499FEF74AFE0446FEF7C3
S31508002D208AFF944908600846008881B292488181E2
S31508002D3034E09148007D002830D18B48C0780128BE
S31508002D4029D188480068FEF7A9FF04468B4A8C4BB0
S31508002D50FEF7CCFF1CD283480068FEF79FFF0446A7
S31508002D60884A894BFEF7AEFF12D281497D48006832
S31508002D70FEF777FE0446FEF75EFF81B27A4810300A
S31508002D8081810146888902F05BFD02F0CBF902E0F9
S31508002D90022002F0BBFD0021734881737248C07B94
S31508002DA0012804D102F0BEF900216F48C1737249A7
S31508002DB08889FEF739FF75490860684908687449C3
S31508002DC0FEF74FFE0746FEF769FF724A724B0191FE
S31508002DD00090FEF7C1FE0446FEF742FF81B2664840
S31508002DE04181FF38C1380088FF21F531884272DDFC
S31508002DF000205D49343908805B48C07801283ED1F7
S31508002E005D48007D00283AD0544988686049FEF735
S31508002E1028FE0446FEF70FFF85B2504948685C490C
S31508002E20FEF71FFE0446FEF706FF80B2854210D164
S31508002E304D483438C068AF218900884209D94E48C0
S31508002E404079002805D148493439C86004214A48E0
S31508002E504171424988680021FEF75CFF05D03F4969
S31508002E6048680021FEF756FF09D1434840790028F3
S31508002E7005D13D493439C86005213F484171374974
S31508002E80C868FEF70BFF0446444A454BFEF71AFF8F
S31508002E9022D23249C868FEF701FF0446414A424B2E
S31508002EA0FEF710FF13D220214048FFF7B9FE00288D
S31508002EB00DD131480079012809D12F4840790028D9
S31508002EC005D129493439C86006212B4841710121A9
S31508002ED02548417011E038E02049C8683449FEF7B2
S31508002EE023FF0AD22448007D002803D100211E486A
S31508002EF0417002E001211C4841701849C8682D49F3
S31508002F00FEF712FF03D201211748017102E00021E2
S31508002F101548017114484078002810D116480079E0
S31508002F20012805D1C1020920C006FFF781FE0CE081
S31508002F300121C9020920C006FFF77CFE05E0012130
S31508002F40C9020920C006FFF775FE07B0F0BD0000EC
S31508002F507001002000F07F450000A0400804002012
S31508002F603333A34048010020B801002000247449E7
S31508002F7000007A4450010020440300206666666615
S31508002F806666E63FCDCCCCCCCCCCEC3F5C030020CF
S31508002F900000C842B81E85EB51B8F63FA245B6F305
S31508002FA0FDD4EC3F75931804560EDD3F0004004827
S31508002FB052B89E3FFCA97940014800687047000056
S31508002FC03C01002003480068034909784018014974
S31508002FD0086070473C0100203401002008B5012133
S31508002FE0480400F085F90121880400F081F9684653
S31508002FF0FFF722FE0421684601804821C170694610
S315080030000920C006FFF77AFD6846FFF715FEFF217F
S315080030100131684601804821C17069460748FFF7B3
S315080030206DFD6846FFF708FE2021684601800421E9
S31508003030C17069460148FFF761FD08BD00040048F4
S3150800304010B504210920C006FFF7EAFD00286CD058
S315080030505B48407A00285DD15948007901283BD160
S315080030605748007D002837D15649C8605648007829
S31508003070401C554908700846007805281FDB0020C3
S3150800308008704F487C38408900280AD14F484D4976
S31508003090C86001214B483430C172FF30113041817C
S315080030A00AE0022147483430C17200204549C86009
S315080030B0002143487C38418101F064F90CE042481C
S315080030C00078022808DC3F48C0687D21090188424B
S315080030D002D900203B49C8603948007D002816D12E
S315080030E03848C0693A49884211D335487C384089FE
S315080030F0002805D137483349C8610020C86006E072
S3150800310031480078022802DC00202E49C8600121D7
S315080031102B4841723048007800280DD101202E49ED
S31508003120087001212648017206E000202A49087025
S315080031300021234801724172224800697D21C90095
S31508003140884237D900201F49086100211C480172AE
S31508003150007D002828D11A487C384088032829DAB7
S3150800316017487C384089002824D11648343000791D
S3150800317000280ED11248007901281BD101211048D8
S31508003180017500200F49C86001210E483430C1720C
S3150800319010E00B48407900280CD1012108484171FC
S315080031A000200849C86005E000200649C8600021DB
S315080031B0034801717E2001F0DDF80148007A10BD50
S315080031C04403002084010020C4000020DC05000020
S315080031D030750000606D00007901002008B50121F6
S315080031E0480400F085F80121880400F081F8684653
S315080031F0FFF722FD402168460180012181701021D8
S31508003200C17069460F48FFF779FC0F496846018087
S31508003210012181701021C17069460920C006FFF797
S315080032206DFC08210920C006FFF704FD20210920AE
S31508003230C006FFF7FFFC10210920C006FFF7FAFCBD
S3150800324008BD00000004004879890000817800293B
S3150800325025D0174903221202891802789210920083
S31508003260895802789207D30EFF229A4091434278F2
S315080032709207120E03789B07DB0E9A4011430C4AFD
S3150800328003231B02D21803789B109B00D1500178A8
S31508003290CA06D20E01219140054A116007E001785D
S315080032A0CA06D20E01219140014A80321160704748
S315080032B000E100E009480A494860002048875A208A
S315080032C088870887074808630020C8620648486256
S315080032D0064888620448C861704700000000344305
S315080032E05C0300209A99993E00002041000048425C
S315080032F0002905D0054A52690243044B5A6104E085
S31508003300024A52698243014B5A61704700100240D3
S31508003310002905D0054AD2690243044BDA6104E064
S31508003320024AD2698243014BDA61704700100240B3
S31508003330002905D0054A92690243044B9A6104E0C4
S31508003340024A92698243014B9A6170470010024013
S3150800335010B500F031F804494968F022114009090E
S31508003360024A515CC84010BD00100240040100200A
S3150800337010B5FFF7EDFF054949680722120211400B
S31508003380090A034A515CC84010BD000000100240FB
S315080033900401002010B5FFF7DBFF0549496807223D
S315080033A0D2021140C90A034A515CC84010BD000048
S315080033B00010024004010020F8B51D4840680C21A1
S315080033C00840042802D008282CD101E0194C2BE02B
S315080033D0174840300069C007C00F09D0144840306C
S315080033E000690221084201D0134802E0114800E0B2
S315080033F0104807460E4840300069FF210904084076
S31508003400000C451C0A48403000690721090208409B
S31508003410000A461C3946694308463146FEF77AFAD9
S31508003420044601E0034C00BF00BF2046F8BD00007B
S315080034300010024000127A0000093D0070B50446EB
S3150800344000250221074800F062FC002808D005483C
S3150800345000F0B4FC20700221024800F050FC01255F
S31508003460284670BD0038014010B500F001F810BDBF
S3150800347000B585B061480068012108435F490860C6
S3150800348000BF5E48006802210842FAD05C485D49E0
S3150800349008605D480068102108435B4908600846D3
S315080034A00068C008C000086056490968481E5749A0
S315080034B0FEF730FA04905448006804994907490F02
S315080034C00843514908604D484068514908404B49EE
S315080034D048600846406890210843484948600846BD
S315080034E040684860474800684549884207D94348C4
S315080034F04068052109020843404948600BE04148F5
S3150800350000684449884206D93C4840680121890236
S3150800351008433A4948606B4601AA3A4801683E485A
S31508003520FEF752FE3548403000698008800033496E
S31508003530403108610846006940084000086168464D
S3150800354000784007400F0290684600794006400E12
S3150800355003902A48C069890508432849C86127484D
S31508003560403000692D4908402449403108610398D4
S3150800357000040299090208432049403109690843B1
S315080035801E49403108611D480068012109060843A3
S315080035901A49086000E000BF18480068012149067A
S315080035A00842F8D0154840688008800013494860EA
S315080035B008464068022108431049486000E000BFF9
S315080035C00E4840680C2108400828F8D10120FEF76B
S315080035D043FF0A484068102188430849486001208B
S315080035E0FEF73AFF0548406880218843034948604A
S315080035F00120FEF731FF05B000BD000000100240B3
S3150800360000A24A04140100200020024000366E0180
S315080036100FC0FFFF0051250200127A00FFF800FFD5
S31508003620042806D10649096904221143044A11618E
S3150800363005E00349096904229143014A116170476B
S3150800364000E000E010B5FFF7BDFC75480088401C97
S31508003650734908800846C068401CC86071480088DD
S31508003660401C7049088070480068002804D06E48DD
S315080036700068401E6C4908606C48007A012805D12C
S3150800368067480069401C6649086102E000206449F1
S31508003690086163483430007A01280ED160484069D1
S315080036A0401C5F494861084640696149884207D914
S315080036B000215B483430017202E000205849486115
S315080036C057483430807A012805D15548C06A401CCD
S315080036D05349C86202E000205149C8625348007D38
S315080036E0002809D04E484068401C4D4948600846A5
S315080036F0806A401C886203E0002049494860886265
S315080037004A48807904280AD14548C0694949884207
S3150800371008D24348C069401C4149C86102E00020FC
S315080037203F49C861FF2101314348FFF779FA00286C
S3150800373013D03B483430407800280ED13B480079F6
S3150800374001280AD13648006A3949884208D23448DD
S31508003750006A401C3249086202E0002030490862CB
S315080037602F483430C07A012813D1C1030920C00676
S31508003770FFF760FA2A4881688068401C284A9060EA
S31508003780FF20F530814225D9002110463430C17218
S3150800379020E023483430C07A022812D18103092058
S315080037A0C006FFF747FA1E4881688068401C1C4A15
S315080037B09060224881420DD9002110463430C172EA
S315080037C008E00020164988600121C9030920C006BF
S315080037D0FFF72EFA1548007D012805D11048006B21
S315080037E0401C0F49086302E000200D4908637E204B
S315080037F000F0C0FD20211048FFF712FA00280AD071
S315080038000748406A0E49884208D20548406A401C63
S315080038100349486202E000200149486210BD0000E1
S3150800382084010020360100203801002044030020CE
S315080038308813000050C3000000040048DC0500009F
S31508003840B888000010B516480068012108431449D5
S315080038500860084640681349084011494860084608
S315080038600068114908400E490860084600680121A9
S31508003870890488430A49086008464068C321090440
S3150800388088430749486008460068084908400449CB
S3150800389008609F2000048860FFF7E6FD10BD000061
S315080038A0001002400CC0FFF8FFFFF6FEFFFF8F0076
S315080038B010B50421080700F017F9002806D00421DE
S315080038C0080700F0EBF801210148817010BD0000DF
S315080038D0B801002008B501214804FFF709FD0222B6
S315080038E001210920C006FFF753F902216846018025
S315080038F01821C1700121817069460920C006FFF7A9
S31508003900FDF808BD10B50121164800F0EDF80028AD
S3150800391027D00121134800F0C1F813488078012800
S315080039201FD11248C179C079401CC2B20F48C27172
S315080039300B2916DD0C48C078012804D1010209209C
S31508003940C006FFF777F90948C0790D2809DD002177
S315080039500548817001210648FEF7FCFB0021034853
S31508003960C17110BD00040040B801002044030020C6
S315080039700024014030B589B004460D4601210846A9
S31508003980FFF7C6FC06A800F047F9079468460583C2
S315080039900021018408A881706846817606A901205D
S315080039A0800700F003F90F21684601710121417172
S315080039B0817101A8FFF74AFC0421080700F06AF89C
S315080039C001220421080700F09AF802A800F0DAF8A4
S315080039D0602168460172012141720020039000218E
S315080039E06846017402A90120800700F093F80821AF
S315080039F0C80600F0BFF84021080600F06DF801215E
S31508003A00880700F03BF80121880700F057F80121E4
S31508003A10880700F047F809B030BD00007FB50446B6
S31508003A200D4601210220FFF773FC684600F0F4F802
S31508003A30019468460580002101818172817069467A
S31508003A400D4800F0B3F8102168460173022141734E
S31508003A500121817303A8FFF7F9FB0121064800F04D
S31508003A6019F801221146044800F049F801210248D4
S31508003A7000F018F87FBD000000040040002904D0BB
S31508003A80026880231A43026003E0026880239A438F
S31508003A900260704702698A430261704702698A4375
S31508003AA002617047002904D0026801231A430260A4
S31508003AB003E002685208520002607047002905D0E8
S31508003AC0426C0123DB031A43426404E0426C01237F
S31508003AD0DB039A4342647047826907231B039A43B0
S31508003AE00B021A438261704702461069084204D0E5
S31508003AF0D068084201D0012070470020FCE7002A60
S31508003B0003D0C3680B43C36002E0C3688B43C3603A
S31508003B107047000010B5826907231B039A430B7888
S31508003B201B021A4382610A7A12014B781B011A4357
S31508003B30036A3024A3431A4302624A6882630C4A22
S31508003B40904213D14A7A12018B781B011A43036AF1
S31508003B50C024A3431A4302624A8992008B899B00B8
S31508003B601A4343682401A3431A43426010BD000068
S31508003B70002C014082690123DB029A430B021A4397
S31508003B808261704700210170417081704160017245
S31508003B90417241818181704701229207904201D189
S31508003BA0816301E08AB282637047000002680323DA
S31508003BB01B029A430B891A430260134A904206D0A5
S31508003BC001229207904202D0104A904205D102681B
S31508003BD070239A438B781A4302600B4A904205D0A9
S31508003BE00B4A904202D00B4A904205D1026B120A48
S31508003BF012028B7A1A4302634A68C2620A88826290
S31508003C000122426170470000002C01400004004078
S31508003C1000440140004801400021C9434160002199
S31508003C200180018181708172704710B5FFF7C4F970
S31508003C3010BD000070B5FFF78BFB05467D21C90056
S31508003C40FDF768FE0446601E0C49884200D90CE060
S31508003C50601E0B4948610321081F00F0E1FB0020A4
S31508003C60074988610720086100BF0420FFF7D8FCD0
S31508003C700021481E00F0D4FB70BD0000FFFFFF00C6
S31508003C8000E000E010B502210A4800F048F80028D4
S31508003C900ED0084800F092F8C4B20748407A0028C7
S31508003CA002D1204601F08CFA0221024800F027F8DA
S31508003CB010BD000000380140B801002010B50446C8
S31508003CC02146054800F07EF800BF0121024800F0B1
S31508003CD01EF80028F9D010BD0038014070B504461A
S31508003CE00D467E2000F046FB03E02078641CFFF7B3
S31508003CF0E5FF2846691E8DB20028F6D170BD4161E0
S31508003D0070478269520852000A4382617047024628
S31508003D109068084201D0012070470020FCE702465F
S31508003D20D068084201D0012070470020FCE7002A2D
S31508003D3003D003690B43036102E003698B43036104
S31508003D407047000070B504460D460026E06930212C
S31508003D50884329790843E061E06944218843A979C1
S31508003D600843E061E06980088000297A0843E06139
S31508003D70A0691821884369890843A061A0690421BC
S31508003D808843297B0843A0610B48844203D1FFF787
S31508003D9001FB064602E0FFF7EBFA064630462968BD
S31508003DA0FDF7B8FD0009206230462968FDF7B2FD27
S31508003DB00007000F606270BD003801400146486880
S31508003DC0C0B27047CAB2026070474B21C901016090
S31508003DD03021017100218171017218214181002170
S31508003DE00173704710B51D484088030000F009FBB1
S31508003DF00504111E2B2C2D0018487C304089FF2104
S31508003E008A31884204DC01211448418000F0BAFA5C
S31508003E101BE012487C304089FF216F31884204DC60
S31508003E2002210E48418000F0ADFA0EE00B487C30C6
S31508003E304089FF215531884204DC03210748418027
S31508003E4000F0A0FA01E000E000BF00BF03487C30A4
S31508003E500079002801D100F095FA10BDC8020020AB
S31508003E6010B576484088002806D0012847D0022891
S31508003E7075D0032842D19DE0022170487C308171BB
S31508003E8020216F48FEF7CCFE002828D06D49C86867
S31508003E90FF21F531FDF73EFDC007C00F0FD11021F8
S31508003EA00920C006FEF7C4FE08210920C006FEF751
S31508003EB0BFFE20210920C006FEF7BAFE1EE010212B
S31508003EC00920C006FEF7B6FE08210920C006FEF73F
S31508003ED0B1FE20210920C006FEF7ACFE0EE0102137
S31508003EE00920C006FEF7A4FE08210920C006FEF731
S31508003EF09FFE20210920C006FEF79AFE9BE00121BD
S31508003F004E487C30817120214D48FEF789FE0028F5
S31508003F1014D04C49C868FF21F531FDF7FBFCC007F2
S31508003F20C00F05D108210920C006FEF781FE0AE068
S31508003F3008210920C006FEF77DFE04E008210920B5
S31508003F40C006FEF775FE10210920C006FEF772FEB0
S31508003F5020210920C006FEF76DFE6CE0FFE7202150
S31508003F603748FEF75DFE002814D03649C868FF2199
S31508003F70F531FDF7CFFCC007C00F05D11021092088
S31508003F80C006FEF757FE0AE010210920C006FEF714
S31508003F904FFE04E010210920C006FEF749FE08215D
S31508003FA00920C006FEF746FE20210920C006FEF7B6
S31508003FB041FE40E020212248FEF732FE002814D0B8
S31508003FC02049C868FF21F531FDF7A4FCC007C00FDA
S31508003FD005D110210920C006FEF72CFE20E010218D
S31508003FE00920C006FEF724FE1AE01649C868CD2146
S31508003FF0FDF790FCC007C00F05D110210920C006A7
S31508004000FEF718FE0CE00F49C868CD21FDF782FCC3
S31508004010C007C00F04D010210920C006FEF708FE0D
S3150800402008210920C006FEF705FE20210920C00642
S31508004030FEF700FE00BF00BF10BD0000C80200204A
S31508004040000400488401002010B5B14880790300B7
S3150800405000F0D7F90504447ED1FDFC00AC48408940
S31508004060FF218A31884203DB0121A948817134E0A6
S31508004070A7484089FF21873188420ADAA4487C3854
S315080040804088022805D00221A1487C38418000F0EA
S3150800409079F920219F48FEF7C3FD00281DD09E49C7
S315080040A0C868FF21F531FDF735FCC007C00F05D1FB
S315080040B010210920C006FEF7BDFD04E010210920E5
S315080040C0C006FEF7B5FD20210920C006FEF7B2FDA1
S315080040D008210920C006FEF7ADFD17E18C48408986
S315080040E0FF21A231884203DB0221894881712EE033
S315080040F020218848FEF794FD002828D08649C868FC
S31508004100FF21F531FDF706FCC007C00F05D10821D0
S315080041100920C006FEF78EFD04E008210920C00626
S31508004120FEF786FD10210920C006FEF783FD202133
S315080041300920C006FEF77EFD75487C3840880128B0
S3150800414005D0012172487C38418000F01BF9DDE07A
S315080041506F484089FF21A531884203DB03216C485B
S31508004160817147E020216B48FEF75AFD002841D0AF
S31508004170FF2101316748FEF753FD002807D066483E
S31508004180006A6649884202D90421614881716249F8
S31508004190C868FF21F531FDF7BDFBC007C00F0FD179
S315080041A010210920C006FEF743FD08210920C00694
S315080041B0FEF73EFD20210920C006FEF739FD0EE078
S315080041C010210920C006FEF735FD20210920C0066A
S315080041D0FEF730FD08210920C006FEF72BFD4C48E6
S315080041E07C384088002805D0002149487C38418021
S315080041F000F0C8F88AE020214648FEF711FD00289D
S3150800420044D0FF2101314348FEF70AFD002807D0B4
S315080042104148006A4149884202D904213C488171D3
S315080042203D49C868FF21F531FDF774FBC007C00F8B
S3150800423012D110210920C006FEF7FAFC0821092030
S31508004240C006FEF7F5FC2021092001E05DE01EE02E
S31508004250C006FEF7EDFC0EE010210920C006FEF7A9
S31508004260E9FC20210920C006FEF7E4FC0821092004
S31508004270C006FEF7DFFC26487C384088002805D0B3
S31508004280002123487C38418000F07CF83EE020215C
S315080042902048FEF7C5FC002836D01D487C384088E3
S315080042A0002805D000211A487C38418000F06AF8B9
S315080042B01948C0691A4988420FD210210920C00638
S315080042C0FEF7B6FC08210920C006FEF7B1FC20213E
S315080042D00920C006FEF7ACFC0EE010210920C00636
S315080042E0FEF7A8FC20210920C006FEF7A3FC08213A
S315080042F00920C006FEF79EFC07483430407801289E
S3150800430002D103210248817100E000BF00BF10BD41
S315080043104403002000040048840100209411000092
S315080043203075000010B5FEF799FAFEF7F5F901F0B9
S31508004330DBFC10BD034880684008400001498860DE
S3150800434070470000002C004003488068002801D010
S31508004350012070470020FCE7002C004010B5FFF74D
S31508004360F3FF002804D0FFF7E5FF662000F002F807
S3150800437010BD00004106490E014A11607047000051
S31508004380002C004010B57E20FFF7F4FF0948FEF721
S31508004390DBFA0949094881800621001D00F0DAF890
S315080043A00649091D8881402202490448001DFEF776
S315080043B008FB10BD00F80008FBAA0000C402002094
S315080043C010B5024A024900F076F810BD9D51000862
S315080043D0800100202021020C01D010211046020A7B
S315080043E001D008391046020901D0091F1046820873
S315080043F001D0891E1046420801D0881E7047081A47
S31508004400704730B47446641E2578641CAB4204D3E6
S31508004410635D5B00E31830BC18471D46F8E70000EB
S3150800442010B5002819DB1A4A03231B02D218830881
S315080044309B00D2588307DC0EFF23A3409A438B07C1
S315080044401B0E8407E40EA3401A43114B03242402CF
S315080044501B198408A4001A5118E00E4A03071B0FFB
S31508004460083B9B089B00D2588307DC0EFF23A3401A
S315080044709A438B071B0E8407E40EA3401A43054B89
S315080044800407240F083CA408A4001A5110BD000014
S3150800449000E100E01CED00E002E008C8121F08C1B8
S315080044A0002AFAD170477047002001E001C1121FA7
S315080044B0002AFBD17047F8B516460F460446002574
S315080044C003E03946B0476D1C641C20780028F8D1F3
S315080044D02846F8BD10B51948007801282DD10020C6
S315080044E0164908701649088012E0154800884000E9
S315080044F01449085A14490988C900144A8918104ADF
S315080045001288520088520E480088401C0C490880C0
S315080045100B4800880428E8DB7E20FFF72BFF0A48B3
S315080045200088401C0849088008460088142804DBCF
S315080045300020088001200649087010BD44010020AB
S315080045405A010020E00300205C0100201804002026
S315080045507801002010B502460023002901D1002069
S3150800456010BD03E01488921CE01883B208464C1E5E
S31508004570A1B20028F6D11846F2E7000070B500256A
S31508004580A648807A01280ED1A4483438C06AFF218B
S31508004590F531884207D90021A04881720020A04938
S315080045A00880A04908709D48407A012870D19C4827
S315080045B0007A012811D003280ED19B48007D0028D7
S315080045C006D19648007A002802D101219348017243
S315080045D0002092493439486119E19148407A072800
S315080045E07ED007DC0300FFF70CFF07122356837EF5
S315080045F093947E000A2874D004DC082872D009280F
S3150800460071D1AEE0A1286FD0A528F9D1F9E0002034
S3150800461082493439486101218048C171002202214A
S315080046208248FFF784FB00207C493439C860ECE0F7
S3150800463000207A49343948617948807A012811D1AD
S315080046407748007B282825DA7548007B0A2821DD6B
S315080046507348017B714810304181012110388173FC
S31508004660C17017E06E48807A022812D16C4A117B15
S31508004670D07A00F063FE0546282D0BDA0A2D09DDEF
S31508004680664810304581012110388173C17001E0F8
S31508004690C1E070BDB9E0002060493439486160481E
S315080046A0807A022823D15E4A117BD07A00F046FE32
S315080046B0012803D103215C48017518E0584A117B8B
S315080046C0D07A00F03BFE002811D10021564801752A
S315080046D05248C07B01280AD100F024FD002104E0DD
S315080046E027E085E035E08FE088E04C48C1738CE030
S315080046F04B48807A02280AD1494A117BD07A00F0C1
S315080047001DFE46491031C88001214448C1737CE02A
S315080047107BE00020414934394861414A117BD07A0F
S3150800472000F00CFE3D4910314880012001F0EEF8FA
S315080047306BE00020394934394861394A117BD07A0F
S3150800474000F0FCFD354910318880032001F0DEF8C1
S315080047505BE00020314934394861022001F0D6F87F
S3150800476053E000202D49343948612D49887AC1170C
S31508004770890F091889108900411A33D12849887A7E
S31508004780C117890F09188910244A10321181104659
S3150800479000891C2826DA00241FE0A200921D204B5F
S315080047A09B1D995CA200521D985C00F0C7FD01464E
S315080047B0A2001A481E308152A2000832184B9B1DCF
S315080047C0995CA200D21D985C00F0B8FD0146A200D3
S315080047D012481E3010184180641C10481030008999
S315080047E0A042DADC042001F091F800F09BFC0CE012
S315080047F0052001F08BF800F095FC06E001F04CF876
S3150800480003E000F0E5FF00E000BF00BF00BF00BF07
S3150800481000210248417200BF3BE70000B8010020B2
S31508004820B80400207C010020440300200038014021
S3150800483070B505460C46002D02D0012D1ED10CE0A0
S31508004840602101208007FFF747F900210120800732
S31508004850FFF7A2F90A48047010E009480078A04258
S3150800486009D0602101208007FFF736F9214601208B
S315080048708007FFF791F90248047000BF00BF70BDBA
S315080048807A01002010B5FE48007901287ED1FD483E
S31508004890007D0028FAD1FA4840790300FFF7B1FDF8
S315080048A008050764BFFEFDFCFBFA002010BDF549AC
S315080048B02039C868FF219131FDF72CF88007800F51
S315080048C00AD110210920C006FEF7B4F908210920EB
S315080048D0C006FEF7AFF940E0EA492039C868FF216B
S315080048E09131FDF717F88007800F01280AD11021AA
S315080048F00920C006FEF79CF908210920C006FEF724
S3150800490099F92AE0DF492039C868FF219131FDF776
S3150800491001F88007800F02280AD110210920C00655
S31508004920FEF788F908210920C006FEF783F914E086
S31508004930D4492039C868FF219131FCF7EBFF80077D
S31508004940800F032809D108210920C006FEF770F94F
S3150800495010210920C006FEF76DF920210920C0069E
S31508004960FEF768F90120A1E7C6492039C868C821B9
S31508004970FCF7D0FF8007800F0CD110210920C00654
S31508004980FEF758F908210920C00600E084E1FEF781
S3150800499051F93DE0BB492039C868C821FCF7BAFF80
S315080049A08007800F01280AD110210920C006FEF7CA
S315080049B03FF908210920C006FEF73CF928E0B1496D
S315080049C02039C868C821FCF7A5FF8007800F022890
S315080049D00AD110210920C006FEF72CF90821092062
S315080049E0C006FEF727F913E0A6492039C868C8218A
S315080049F0FCF790FF8007800F032809D108210920BA
S31508004A00C006FEF715F910210920C006FEF712F9AF
S31508004A1020210920C006FEF70DF9012046E799492D
S31508004A202039C868C821FCF775FF8007800F0AD1AE
S31508004A3010210920C006FEF7FDF808210920C00646
S31508004A40FEF7F8F843E08F492039C868C821FCF713
S31508004A5061FF8007800F01280AD110210920C006AE
S31508004A60FEF7E6F808210920C006FEF7E3F82EE06F
S31508004A7084492039C868C821FCF74CFF8007800F95
S31508004A80022810D110210920C006FEF7D3F8082104
S31508004A90092004E0FFE0D0E076E04AE01EE0C00628
S31508004AA0FEF7C8F813E077492039C868C821FCF72B
S31508004AB031FF8007800F032809D108210920C00685
S31508004AC0FEF7B6F810210920C006FEF7B3F8202134
S31508004AD00920C006FEF7AEF80120E7E66949203945
S31508004AE0C868FF212D31FCF715FFC007C00F05D197
S31508004AF010210920C006FEF79DF80EE0614920390D
S31508004B00C868FF212D31FCF705FFC007C00F04D088
S31508004B1010210920C006FEF78BF820210920C006BF
S31508004B20FEF788F808210920C006FEF783F8012059
S31508004B30BCE654492039C868FF219131FCF7EAFEE2
S31508004B40C007C00F05D110210920C006FEF772F86C
S31508004B500EE04C492039C868FF219131FCF7DAFE8E
S31508004B60C007C00F04D010210920C006FEF760F860
S31508004B7020210920C006FEF75DF808210920C00695
S31508004B80FEF758F8012091E63E492039C868C82141
S31508004B90FCF7C0FE8007800F0AD110210920C00645
S31508004BA0FEF748F808210920C006FEF743F83DE05D
S31508004BB034492039C868C821FCF7ACFE8007800F45
S31508004BC001280AD110210920C006FEF731F808216C
S31508004BD00920C006FEF72EF828E02A492039C868B9
S31508004BE0C821FCF797FE8007800F02280AD11021FA
S31508004BF00920C006FEF71EF808210920C006FEF7A0
S31508004C0019F813E01F492039C868C821FCF782FE45
S31508004C108007800F032809D108210920C006FEF75E
S31508004C2007F810210920C006FEF704F820210920FC
S31508004C30C006FDF7FFFF012038E612492039C8688B
S31508004C40C821FCF767FEC007C00F05D1102109204F
S31508004C50C006FDF7EFFF0DE00A492039C868C821EC
S31508004C60FCF758FEC007C00F04D010210920C00663
S31508004C70FDF7DEFF20210920C006FDF7DBFF03E074
S31508004C8044030020A401002008210920C006FDF7DE
S31508004C90D1FF01200AE600BF00BF07E610B5F648B7
S31508004CA0007D002833D0F548C07801282FD1F34875
S31508004CB03438C068F24988420ED9EF48808964289A
S31508004CC00ADAED484079002806D10721EA484171F9
S31508004CD00020EA493439C860E748007D032816D021
S31508004CE0E5488089FF21EB31884210DDE2484079AA
S31508004CF000280CD1E1483438C068E249884206D910
S31508004D000321DD4841710020DC493439C860DA489E
S31508004D10007901286FD1D84840790300FFF771FB65
S31508004D20080507427EB8F7EFEEED002010BDD34820
S31508004D303438C068E121C90088422DD908210920E4
S31508004D40C006FDF777FF20210920C006FDF772FF90
S31508004D5010210920C006FDF76DFF0121C748143848
S31508004D60017514308079002807D1C4493439C860E0
S31508004D700021C148017141710AE0C0483438C06851
S31508004D80AF210901884203D90020BC493439C860DB
S31508004D900121BA48417103E00021B8481438017569
S31508004DA00120C3E7B5483438C068B74988422FD9C7
S31508004DB008210920C006FDF73DFF20210920C0066D
S31508004DC0FDF738FF10210920C006FDF733FF012142
S31508004DD0AA48143801751430807900280CD1A749DF
S31508004DE03439C8600021A448017141710020A349E3
S31508004DF03439C86010E03DE1A0483438C068AF21B6
S31508004E000901884208D900209C493439C86003E062
S31508004E1000219A4814380175012087E797483438E5
S31508004E20C0689A4988422DD908210920C006FDF78D
S31508004E3001FF20210920C006FDF7FCFE10210920EC
S31508004E40C006FDF7F7FE01218C48143801751430A9
S31508004E50807900280BD189493439C86000218648F1
S31508004E6001714171002085493439C8600EE08348D4
S31508004E703438C0688649884208D900207F493439C1
S31508004E80C86003E000217D481438017501204DE70C
S31508004E907A483438C0687D210901884231D9082109
S31508004EA00920C006FDF7C6FE20210920C006FDF729
S31508004EB0C1FE10210920C006FDF7BCFE01216F487E
S31508004EC0143801751430807900280BD16B493439B0
S31508004ED0C86000216848017141710020674934396A
S31508004EE0C86012E065483438C068664988420CD9FB
S31508004EF0002062493439C86007E0BAE07EE042E043
S31508004F0005E000215D481438017501200EE75B486D
S31508004F103438C068E121C90088422ED90821092001
S31508004F20C006FDF787FE20210920C006FDF782FE90
S31508004F3010210920C006FDF77DFE01214F481438CF
S31508004F4001751430807900280BD14C493439C86072
S31508004F500021494801714171002048493439C86027
S31508004F600FE046483438C068AF210901884208D99D
S31508004F70002042493439C86003E000213F4814380C
S31508004F8001750120D2E63D483438C0684049C83921
S31508004F9088422DD908210920C006FDF74BFE20219D
S31508004FA00920C006FDF746FE10210920C006FDF7B8
S31508004FB041FE0121314814380175143080790028E2
S31508004FC00BD12E493439C86000212B480171417133
S31508004FD000202A493439C8600EE028483438C068A9
S31508004FE02C49884208D9002024493439C86003E08E
S31508004FF00021224814380175012097E61F483438E5
S31508005000C068214988422ED908210920C006FDF723
S3150800501011FE20210920C006FDF70CFE10210920EB
S31508005020C006FDF707FE012114481438017514302F
S31508005030807900280BD111493439C86000210E48FF
S315080050400171417100200D493439C8600FE00B48E1
S315080050503438C0680D49C831884208D90020074944
S315080050603439C86003E0002104481438017501206A
S315080050705CE600BF00BF59E644030020B8010020E3
S31508005080204E0000B80B0000A4060000C40900006A
S31508005090AC0D0000CC10000010B5052416E0FF2169
S315080050A001311F48FCF779FCFF2101311C48FDF747
S315080050B0B3FAFE211A48FDF7B3F901461848E0305D
S315080050C0C08B814202D100F065FB10BD2046611EEF
S315080050D0CCB20028E3D1052416E0FF21013110489F
S315080050E0FCF75BFCFF2101310D48FDF7B3FAFE2101
S315080050F00B48FDF795F901460948E030C08B814217
S3150800510002D100F047FBE0E72046611ECCB200283A
S31508005110E3D100F03DF900F005F800BFD5E700003F
S31508005120C801002010B5FDF7F9FB1A491A48818015
S31508005130001D00891C2815DA1748001D01890E3044
S31508005140FDF7E8F81449091D088908E000228300DC
S3150800515011491231CA52830059184A80401C1E2828
S31508005160F4D300E010BDFE210B48001DFDF758F9E9
S3150800517001460948E430C183FF210131E038FDF7D3
S31508005180A5FAFF2101310448001DFDF7ABFA00BF5F
S31508005190E8E70000FBAA0000C401002070B5044639
S315080051A00D46E1B20548FEF70DFE00BF0121034892
S315080051B0FEF7ADFD0028F9D0204670BD0038014045
S315080051C070B50446002501215948817200205849C6
S315080051D03439C86257480088FA2804DD0020554942
S315080051E0088055490870544800780300FFF709F904
S315080051F008051D2B3F4B586D799CAA2C0DD1012013
S315080052004D4908704B4801880088401C494A10805F
S31508005210901D445400201146C870BB2C04D10121AE
S315080052200920C006FDF704FD7FE0FB2C0AD14148A2
S3150800523001880088401C3F4A1080901D4454022073
S315080052403D49087071E0012C03D103203A490870E2
S3150800525004E0032C02D10620374908703548018836
S315080052600088401C334A1080901D44545DE0314844
S3150800527001880088401C2F4A1080901D4454042041
S315080052802D49087051E02B48847001880088401C1D
S31508005290284A1080901D445405202749087044E088
S315080052A02448C078401CC0B22249C8708978884210
S315080052B002DB0620204908701E4801880088401C29
S315080052C01C4A1080901D44542FE01A480188008813
S315080052D0401C184A1080901D44540720164908702F
S315080052E023E0144801880088401C124A1080901D4B
S315080052F04454801F0188801DFDF792F8002809D1C3
S3150800530000210B4881720121417200200A49087068
S315080053100849088007480088FA2804DD002005495E
S3150800532008800549087000E000BF00BF70BD000096
S31508005330B8010020B80400207C01002070B50246A0
S31508005340002013460C461D02FF263602354025432B
S31508005350284670BD00BF00BF00BF00BF00BF00BF2A
S3150800536000BF00BF00BFFEE707490848818000214B
S31508005370001D41805F21C900C180152181805F2100
S315080053800181002141817047FBAA0000C402002068
S3150800539000201D4A1D498A80F022091D4A801422D0
S315080053A08A8002220A8119224A81194A8A81920030
S315080053B0CA8000BF0FE00022830014498A31CA520E
S315080053C0830059184A80830010491231CA52830053
S315080053D059184A80401C1C28EDDB00220B49091D80
S315080053E0CA81FF225F320A8214224A82FF225F3272
S315080053F08A8200228031CA80891D4A8014228A80C6
S31508005400FF225F32CA807047FBAA0000C401002051
S31508005410EE02000010B57E20FEF7ACFFFFF732FA69
S31508005420012800D110BD5F48007901287ED15D486A
S31508005430007D002802D001285DD133E020215A489A
S31508005440FDF7EEFB002822D15848C0695849884222
S3150800545027D25648C0687D210901884221D2514881
S315080054607C384089002802D1FEF7FAFC19E01021A1
S315080054700920C006FDF7DEFB20210920C006FDF73E
S31508005480D9FB08210920C006FDF7D4FB09E04748E7
S31508005490406A4749884202D2FEF7E2FC01E0FEF77D
S315080054A0D3FD7BE04149C868FF21F531FCF732FAA4
S315080054B0C007C00F0FD110210920C006FDF7B8FBA1
S315080054C008210920C006FDF7B3FB20210920C006E4
S315080054D0FDF7AEFB0EE010210920C006FDF7AAFB7A
S315080054E020210920C006FDF7A5FB08210920C006D2
S315080054F0FDF7A0FB52E02B48007D05282AD12B4951
S31508005500C868FF21F531FCF705FAC007C00F11D1AD
S3150800551010210920C006FDF78BFB08210920C006CB
S31508005520FDF786FB20210920C00600E037E0FDF7DD
S315080055307FFB32E010210920C006FDF77BFB202106
S315080055400920C006FDF776FB08210920C006FDF7ED
S3150800555071FB22E01348007D06280FD1102109208F
S31508005560C006FDF767FB20210920C006FDF762FB90
S3150800557008210920C006FDF75DFB0EE01021092071
S31508005580C006FDF755FB08210920C006FDF750FBAC
S3150800559020210920C006FDF74BFB00BF00BF00BF56
S315080055A040E700004403002000040048840100206E
S315080055B030750000FEF746F9FDF710FE08210920B0
S315080055C0C006FDF737FB20210920C006FDF732FB90
S315080055D010210920C006FDF72DFBE1204002FCF74B
S315080055E0C9FEFDF7FBFCFCF76FFFFCF70FFD0C206F
S315080055F0FCF77AFC0920FCF777FC0820FCF774FC1A
S315080056000720FCF771FC01214848FCF7A3FD01219E
S315080056104748017100214171FF388D384171817108
S31508005620012143484172FDF70BFDFEF753F9414945
S315080056306320FEF79FF91A216320FEF7EFF9FFF7BB
S315080056402BFDFEF7F7FA00F07FF839487C384089D9
S31508005650002801D1FEF704FC00213748417040219B
S315080056600920C006FDF7E6FA40213448FDF7E2FABC
S31508005670FEF758FE00213048C171FDF71BFE0121D7
S315080056800920C006FDF7D6FA4EE02B48C079002857
S3150800569002D0012843D10AE0FEF770FFFCF782FD2D
S315080056A0FFF7B8FEFDF7CCFC00F044FB3BE0002119
S315080056B0084600F057F920483438C068204988421F
S315080056C008D900211C48C171012202211D48FEF794
S315080056D02EFB1EE018493439C868FF21F531FCF75E
S315080056E019F9C007C00F0FD110210920C006FDF710
S315080056F0A1FA20210920C006FDF79CFA08210920F5
S31508005700C006FDF797FA04E020210920C006FDF738
S315080057108FFAFCF7ABFD7E20FEF72CFE03E0002196
S315080057200548C17100BF00BFAFE700000024014073
S3150800573044030020581B0000B8010020000400485C
S31508005740204E00000038014010B540210F48FCF7F4
S3150800575024F940210D48FCF79BFF06210B48FEF76C
S31508005760F9FE0A49898988420AD10848001F8088B3
S315080057700749884208D0FFF7F7FDFEF703FE03E066
S31508005780FFF7F2FDFEF7FEFD10BD0000C80200207F
S31508005790FBAA000010B500240C484089052803DB45
S315080057A00A484089282803DD19210848418101242F
S315080057B0064800891D2803DD0124022103480181CA
S315080057C0012C01D1FFF7AEFC10BD0000C801002076
S315080057D070B5A0B00025002680216846FCF7DDF8E4
S315080057E0AA2168460170FB21417001218170A5211B
S315080057F0C1701248007A8006010E68460171027966
S315080058000E490E31401DFCF7AFF868460079411D78
S315080058106846FCF705FE0446211268460079401DD5
S315080058206A46115468460079801D14546846007902
S31508005830C11D6846FEF752FA20B070BDC8010020A7
S3150800584030B5A1B00446802101A8FCF7A6F80025CA
S31508005850AA2168460171FB2141710221817101214A
S31508005860C17102210172FF20000220400112684620
S3150800587041728472072101A8FCF7D2FD0546FF2074
S315080058800002284001126846C1720573092101A861
S31508005890FEF724FA21B030BDF0B5A1B000260027E6
S315080058A0802101A8FCF779F80025AA21684601712C
S315080058B0FB21417101218171A121C1710B21017265
S315080058C00FA5027A29460930FCF74EF86846007A91
S315080058D0411D01A8FCF7A4FD044621126846007A7A
S315080058E0401D01AA11546846007A801D1454684662
S315080058F0007AC11D01A8FEF7F1F921B0F0BD00003C
S315080059004E5F433243355F56315F310030B5A1B043
S315080059100446802101A8FCF740F80025AA2168461C
S315080059200171FB214171022181710521C171022199
S315080059300172FF20000220400112684641728472FB
S31508005940072101A8FCF76CFD0546FF200002284048
S3150800595001126846C1720573092101A8FEF7BEF94E
S3150800596021B030BD70B504460D460026002D13D172
S315080059700846FEF75DFF0021D4480182FF388D38BE
S3150800598041730020D2498862D2490870D049086319
S315080059900021CE48418297E1CD483430407B00282B
S315080059A077D1CB48806AFF21F531884272D9002029
S315080059B0C7498862C5488189601F81420EDDC5488E
S315080059C00078C54908600221C14834304173BF4890
S315080059D0818901827D20C000C0490880BB48018AB0
S315080059E0808981420BDD0121B94834304173B748BB
S315080059F0818901827D20C000B84908800EE0B3483D
S31508005A00818920461430814208DDB24800780F2883
S31508005A1004DDB0480078401FAE490870AB4881895C
S31508005A2020463738814236DAA8487C38408800282C
S31508005A3003D14820A749087010E0A4487C3840885C
S31508005A40012803D15120A349087007E09F487C38F4
S31508005A504088022802D15A209E4908709C48006B4B
S31508005A609F49884230D90020994908639748418A56
S31508005A708089814209DB95484079002805D10721AC
S31508005A809248417100209249C860904881894182B4
S31508005A901AE022E01BE08D4881892046263881429B
S31508005AA009DD8C4800780F280EDD8A480078801EAC
S31508005AB08849087008E0874800780F2804DD85487B
S31508005AC00078C01E83490870804881890182814810
S31508005AD001780120FEF7ACFEF6E07D483430407BC5
S31508005AE001287CD17A48806A7C490988884262D92B
S31508005AF00020774988627548018A808981425BDA85
S31508005B007248818920461438814215DAFF20F5301B
S31508005B10724908806D488189008A081A042805DABE
S31508005B206C480078801C6B49087035E06948007835
S31508005B30401C684908702FE06448818920460A3865
S31508005B40814215DAFF20F530644908805F4881896B
S31508005B50008A081A022805DA5E480078401C5D4962
S31508005B60087019E05B480078801E5A49087013E0EF
S31508005B7056488189601F81420EDAFF20F530574961
S31508005B80088052488189008A081A022804DB51488D
S31508005B900078801E4F4908704C48818901828089A7
S31508005BA0A04256DD7D20C0004C490880494800784F
S31508005BB0801E484908704CE044488089A04219DD97
S31508005BC042488089001B05280ADD7D20C00043491C
S31508005BD0088040480078801E3E49087036E04DE04F
S31508005BE07D20C0003D4908803A480078401E394962
S31508005BF008702BE035488089A04227D03348818930
S31508005C00008A081A032805DD32480078801C3149C5
S31508005C1008701BE02D48818920460838814209DA38
S31508005C20AF2080002D4908802A480078C01C2949E1
S31508005C3008700BE02B482949088024488089A0422F
S31508005C4004DA24480078801C224908701F48818994
S31508005C500182204800780A2803DA0A201D490870BC
S31508005C6006E01C4800783C2802DD3C2019490870EB
S31508005C70184801780120FEF7DBFD25E01548007875
S31508005C80282804DD134800781038124908700F4890
S31508005C908189E01C814204DC0C488189E01E81422E
S31508005CA00ADA01210A483430417308488189018299
S31508005CB07D20C00009490880044881890182054879
S31508005CC001780120FEF7B4FD70BD000044030020F2
S31508005CD084010020EE000020F4000020F0000020DF
S31508005CE0B80B0000DC05000008B501214804FDF7E3
S31508005CF0FFFA01218804FDF7FBFA6846FCF79CFFCA
S31508005D000421684601804821C17069460920C006F9
S31508005D10FCF7F4FE6846FCF78FFF202168460180F1
S31508005D200421C17069460248FCF7E8FE08BD000078
S31508005D300004004810B50024FEF7B0FF01280CD176
S31508005D40E948C068FF21F531884205D90121C90310
S31508005D500920C006FCF76CFF10BDE448007900284E
S31508005D607BD1E349087000210846FFF7FBFD0021B7
S31508005D70DD483430C1701438017508210920C00681
S31508005D80FCF758FF20210920C006FCF753FF102115
S31508005D900920C006FCF74EFF0021D4480175D248F9
S31508005DA0C068FF21F531884209D2CF48343040799E
S31508005DB0002803D10121CC483430C17286E1002184
S31508005DC0C948343041713438C068CA49884235D91F
S31508005DD0C648407A002812D1C348C0687D214901C7
S31508005DE0884204D2C4A0FEF7EBFAFDF7FBFF0021B8
S31508005DF0BE4841717D204001BB49C8600CE0BB48E4
S31508005E00007A012808D10020B749C8600021B748A0
S31508005E1041710175012101712021B848FCF700FF85
S31508005E20002805D00021B1480175012101714DE115
S31508005E3001210920C006FCF7FBFE47E1AB48007AC2
S31508005E400128BBD10020A849C8600021A748417194
S31508005E5001750121017139E1FFE7A448007D0300BE
S31508005E60FEF7CFFA07056182A4AEB7EF60000021FE
S31508005E700846FFF777FD9C483430807B002804D11C
S31508005E80002199483430C17003E001219648343026
S31508005E90C17095483430C07B012805D1FFF742F917
S31508005EA0002191483430C1738F48C0687D210901AB
S31508005EB0884228D900208E4908708B483430007AE9
S31508005EC000282FD120218D48FCF7AAFE002816D1DC
S31508005ED008210920C006FCF7ADFE20210920C006CE
S31508005EE0FCF7A8FE10210920C006FCF7A3FEFDF763
S31508005EF079FF01210920C006FCF79AFE12E000206E
S31508005F007949C8600EE07848C068FF21F5318842B3
S31508005F1008D976487C384089002803D10021724880
S31508005F203430C172D1E001216F4834304170C170FC
S31508005F306D49C8687D21C900FBF7ECFC6A49443104
S31508005F408988884206D90221684801750121FF38E7
S31508005F508D38C1726449C86800F0D4F80446012136
S31508005F602046FFF7FFFCB0E001215F48343041705E
S31508005F70C1705D49C86800F0C5F80446012120468D
S31508005F80FFF7F0FC5849C8687D21C900FBF7C2FC39
S31508005F905549443149880F39884206D90121524862
S31508005FA03430C1720521514801758EE001214E48F1
S31508005FB034304170C170FF208730FFF7D3FC84E08E
S31508005FC0012149483430C17000210846FFF7CAFC50
S31508005FD07BE0012144483430C1703438C16844300C
S31508005FE04088401E7D22D2005043FF30F530814262
S31508005FF009D23D49C86800F085F8044601212046C3
S31508006000FFF7B0FC44E000210846FFF7ABFC01218E
S3150800601035483430C1723438C16844304088401E2F
S315080060207D22D2005043AF229200801881422FD39E
S315080060302D4834308079012804D106212B48017572
S3150800604020E026E020212D48FCF7EAFD002816D19D
S3150800605008210920C006FCF7EDFD20210920C0060D
S31508006060FCF7E8FD10210920C006FCF7E3FDFDF763
S31508006070B9FE01210920C006FCF7DAFD02E000217D
S315080060801A4801750121C9030920C006FCF7D0FD8D
S315080060901BE016484079002816D11348C0681849ED
S315080060A0884211D9FDF79EFE00200F49C8600F48A7
S315080060B07C384088032803DA01210C48017503E07F
S315080060C000210A480175017100BF00BF06484068F3
S315080060D0FF21F531884202D90020034948607E2015
S315080060E0FEF748F900BF37E6840100204403002084
S315080060F0C4000020B80B000031313100000400480C
S3150800610010270000F8B5054600247D21C900284659
S31508006110FBF700FC064600270020009000BF0BE0B6
S31508006120A1000C48405AB04205DCA10009480818ED
S31508006130408800900127641C06480E380089A04252
S31508006140EEDC002F03D103480E38008A0090009831
S31508006150F8BD0000D601002000C1814001C0804181
S3150800616001C0804100C1814001C0804100C1814019
S3150800617000C1814001C0804101C0804100C1814009
S3150800618000C1814001C0804100C1814001C08041F9
S3150800619001C0804100C1814001C0804100C18140E9
S315080061A000C1814001C0804100C1814001C08041D9
S315080061B001C0804100C1814000C1814001C08041C9
S315080061C001C0804100C1814001C0804100C18140B9
S315080061D000C1814001C0804101C0804100C18140A9
S315080061E000C1814001C0804100C1814001C0804199
S315080061F001C0804100C1814000C1814001C0804189
S3150800620001C0804100C1814001C0804100C1814078
S3150800621000C1814001C0804100C1814001C0804168
S3150800622001C0804100C1814001C0804100C1814058
S3150800623000C1814001C0804101C0804100C1814048
S3150800624000C1814001C0804100C1814001C0804138
S3150800625001C0804100C1814000C0C101C30302C220
S31508006260C60607C705C5C404CC0C0DCD0FCFCE0E88
S315080062700ACACB0BC90908C8D81819D91BDBDA1AF8
S315080062801EDEDF1FDD1D1CDC14D4D515D71716D668
S31508006290D21213D311D1D010F03031F133F3F232D8
S315080062A036F6F737F53534F43CFCFD3DFF3F3EFE48
S315080062B0FA3A3BFB39F9F83828E8E929EB2B2AEAB8
S315080062C0EE2E2FEF2DEDEC2CE42425E527E7E62628
S315080062D022E2E323E12120E0A06061A163A3A26298
S315080062E066A6A767A56564A46CACAD6DAF6F6EAE08
S315080062F0AA6A6BAB69A9A86878B8B979BB7B7ABA78
S31508006300BE7E7FBF7DBDBC7CB47475B577B7B676E7
S3150800631072B2B373B17170B0509091519353529257
S3150800632096565797559594549C5C5D9D5F9F9E5EC7
S315080063305A9A9B5B99595898884849894B8B8A4A37
S315080063404E8E8F4F8D4D4C8C4484854587474686A7
S31508006350824243834181804078630008C800002058
S31508006360BC0000009844000834640008840100203A
S315080063703C080000A84400080000000000000000D7
S3150800638000000000000000000000000000000000FF
S3150800639000000000000000000000000000000000EF
S315080063A000000000000000000000000000000000DF
S315080063B000000000000000000102030401020304BB
S315080063C00607080900A24A040000000000000000B1
S315080063D00102030406070809000000000000000087
S315080063E0040000000100000000000000000000009A
S315080063F0000000000000000000000000000000008F
S31508006400000000000000000000000000000000007E
S31508006410000000000000000000000000000000006E
S31508006420000000000000000000000000000000005E
S30908006430000000005A
S705080018C515
